:100000000C942A000C9445000C9445000C94450077
:100010000C9445000C94BE010C94EB010C941D0251
:100020000C9445000C945C010C9445000C94450024
:100030000C9445000C9442080C943F030C9445002A
:100040000C9445000C9445000C9445000C9445001C
:100050000C94450011241FBECFE5D4E0DEBFCDBF18
:1000600010E0A0E6B0E0EEEDFEE102C005900D92DA
:10007000AC3BB107D9F711E0ACEBB0E001C01D9289
:10008000AE34B107E1F70C94AD000C940000CF93AF
:10009000DF93CDB7DEB7E7E3F0E08FE18083E4E301
:1000A000F0E08EEF8083E1E3F0E084E08083E2E340
:1000B000F0E088E38083DF91CF910895CF93DF93C1
:1000C000CDB7DEB721970FB6F894DEBF0FBECDBF18
:1000D000F89480E29EE490934B0180934A01198248
:1000E0002FC08981482F552789819927880F991F0B
:1000F000FC01E252FF4F808191819C0128513C4FCD
:10010000CA01880F991FFC01E65CFE4F31832083F2
:1001100020914A0130914B0189819927880F991FBD
:10012000FC01E65CFE4F80819181A901481B590BBF
:10013000CA0190934B0180934A0189818F5F898323
:100140008981883070F2789421960FB6F894DEBFDA
:100150000FBECDBFDF91CF910895CF93DF93CDB781
:10016000DEB721970FB6F894DEBF0FBECDBF0E9459
:1001700047000E943A010E9431030E9480031092BE
:1001800039018CED92E09093D9008093D8008AE2F7
:1001900093E09093DB008093DA0078948091C00024
:1001A0008823E1F31092C0000E9429060E9468048F
:1001B0000E94930700C08091CA00813041F4809171
:1001C0003901882311F40E945E001092CA008091C8
:1001D000C300813021F41092C3000E94E707809190
:1001E000C100813011F41092C1008091C0008130B3
:1001F00019F51092C00019821CC080E690E00E94A0
:10020000BA03898199270E94040487E690E00E943E
:10021000BA0389819927880F991FFC01E65CFE4F7C
:10022000808191810E9404040E94F50389818F5F7F
:1002300089838981893008F38091BF00813009F07A
:10024000BACF1092BF000E947006B5CFCF93DF9354
:10025000CDB7DEB7F894E9E5F0E089E180837894E2
:10026000DF91CF910895CF93DF93CDB7DEB7DF91C4
:10027000CF910895CF93DF93CDB7DEB7E3E5F0E0FC
:1002800082E08083EFE4F0E01082EEE4F0E082E0D0
:100290008083EAE4F0E084EF91E091838083E8E4F6
:1002A000F0E080ED97E091838083E9E5F0E081E084
:1002B0008083DF91CF9108951F920F920FB60F9216
:1002C00011248F93CF93DF93CDB7DEB78091CF000A
:1002D0008F5F8093CF008091CF00833029F481E03D
:1002E0008093C3001092CF00809138018F5F80937C
:1002F0003801809138018732C9F581E08093C100CF
:10030000109238018091CE008F5F8093CE00809153
:10031000CE00853029F41092CE0081E08093C20097
:100320008091CC008F5F8093CC008091CC0084368C
:1003300041F41092CC0081E08093BE0081E0809374
:10034000C0008091CC00823319F481E08093C0001A
:100350008091CD008F5F8093CD008091CD008A3059
:1003600029F41092CD0081E08093BF00DF91CF91FE
:100370008F910F900FBE0F901F9018951F920F92A4
:100380000FB60F9211242F933F934F935F936F9368
:100390007F938F939F93AF93BF93EF93FF93CF93ED
:1003A000DF93CDB7DEB7E091D800F091D900099581
:1003B000DF91CF91FF91EF91BF91AF919F918F917D
:1003C0007F916F915F914F913F912F910F900FBE51
:1003D0000F901F9018951F920F920FB60F92112435
:1003E0008F93AF93BF93EF93FF93CF93DF93CDB7EB
:1003F000DEB7A2E3B0E0E2E3F0E080818B7F8C9394
:10040000A5E3B0E0E5E3F0E080818D7F8C9381E0AF
:100410008093C9008091BC00883019F481E08093FA
:10042000CA00DF91CF91FF91EF91BF91AF918F9172
:100430000F900FBE0F901F9018951F920F920FB63E
:100440000F9211242F933F938F939F93AF93BF935A
:10045000EF93FF93CF93DF93CDB7DEB72297DEBF45
:10046000CDBFA2E3B0E0E2E3F0E0808184608C9352
:10047000ECE4F0E011821082A8E4B0E08091BC00CE
:100480009927880F991FFC01E65CFE4F80819181BE
:1004900011969C938E938091BC00882339F4A5E338
:1004A000B0E0E5E3F0E0808182608C938091BC0055
:1004B000282F33273A83298389819A8182309105B5
:1004C000C1F129813A812330310554F489819A811F
:1004D000009789F029813A8121303105D9F04EC049
:1004E00089819A818330910599F129813A8124305B
:1004F0003105E9F143C0A8E3B0E0E8E3F0E0808132
:1005000080618C93A8E3B0E0E8E3F0E08081816053
:100510008C9334C0A8E3B0E0E8E3F0E080818E7F04
:100520008C93A8E3B0E0E8E3F0E0808182608C93F4
:1005300025C0A8E3B0E0E8E3F0E080818D7F8C93F4
:10054000A8E3B0E0E8E3F0E0808184608C9316C01B
:10055000A8E3B0E0E8E3F0E080818B7F8C93A8E330
:10056000B0E0E8E3F0E0808188608C9307C0A8E306
:10057000B0E0E8E3F0E08081877F8C938091BC005D
:100580008F5F8093BC008091BC00893010F0109286
:10059000BC002296F894DEBFCDBFDF91CF91FF91D2
:1005A000EF91BF91AF919F918F913F912F910F90BC
:1005B0000FBE0F901F901895CF93DF93CDB7DEB786
:1005C0008091D0009091D1000097B1F4E6E4F0E082
:1005D000808191819093D7008093D600AEE4B0E003
:1005E000EEE4F0E080818F7B8C9381E090E090934B
:1005F000D1008093D0002BC0E6E4F0E080819181AF
:100600009093D5008093D400AEE4B0E0EEE4F0E047
:10061000808180648C932091D4003091D5008091AA
:10062000D6009091D700A901481B590BCA0190939D
:10063000D3008093D2001092D1001092D00080910C
:10064000D2009091D30090934D0180934C01DF91A3
:10065000CF910895CF93DF93CDB7DEB7DF91CF91E0
:100660000895CF93DF93CDB7DEB7E7E2F0E01082D5
:10067000E6E2F0E08FEE8083DF91CF9108951F9244
:100680000F920FB60F9211242F933F938F939F9346
:10069000EF93FF93CF93DF93CDB7DEB7E6E2F0E0C1
:1006A00010828091BD009927E4E2F0E02081318141
:1006B000880F991FFC01E252FF4F31832083809104
:1006C000BD008F5F8093BD008091BD00873010F02A
:1006D0001092BD00E7E2F0E08091BD008083E6E289
:1006E000F0E08FEE8083DF91CF91FF91EF919F91AA
:1006F0008F913F912F910F900FBE0F901F901895E3
:10070000CF93DF93CDB7DEB7E9E2F0E080E18083FD
:10071000E0E4F0E01082EAE2F0E088E18083E0E4E7
:10072000F0E086E88083EBE2F0E082EC8083DF910A
:10073000CF910895CF93DF93CDB7DEB721970FB652
:10074000F894DEBF0FBECDBF8983EBE2F0E080817D
:100750009927807290700097C1F3ECE2F0E08981F4
:10076000808321960FB6F894DEBF0FBECDBFDF9118
:10077000CF910895CF93DF93CDB7DEB726970FB60D
:10078000F894DEBF0FBECDBF9E838D838D819E8189
:10079000DC01FD0101900020E9F73197CF018A1BB0
:1007A0009B0B9C838B831A8219820FC029813A810B
:1007B0008D819E81F901E80FF91F80810E949A03C3
:1007C00089819A8101969A83898329813A818B81D3
:1007D0009C818217930750F726960FB6F894DEBFD8
:1007E0000FBECDBFDF91CF910895CF93DF93CDB7EB
:1007F000DEB780916A000E949A0380916B000E948C
:100800009A03DF91CF910895CF93DF93CDB7DEB7F1
:1008100066970FB6F894DEBF0FBECDBF9E8B8D8B53
:100820008D899E894AE050E09E012F5F3F4FB901BC
:100830000E94F30ECE0101960E94BA0366960FB68F
:10084000F894DEBF0FBECDBFDF91CF910895CF9357
:10085000DF93CDB7DEB722970FB6F894DEBF0FBE99
:10086000CDBF8A8387E089831FC08A81482F55279F
:100870008981282F332727FD309581E090E0022ED3
:1008800002C0880F991F0A94E2F784239523181653
:10089000190624F481E30E949A0303C080E30E94B6
:1008A0009A0389818150898389818823F4F6809114
:1008B0006A000E949A0380916B000E949A0322961C
:1008C0000FB6F894DEBF0FBECDBFDF91CF91089574
:1008D000CF93DF93CDB7DEB70E94A10463E080E041
:1008E0000E9405068CE690E00E94A70562E081E088
:1008F0000E94050687E790E00E94A7050E949704E2
:10090000E0E3F0E080819927807290700097C1F752
:100910000E94A104DF91CF910895CF93DF93CDB7CB
:10092000DEB78DE00E94DC05DF91CF910895CF9373
:10093000DF93CDB7DEB78CE00E94DC05DF91CF916D
:100940000895CF93DF93CDB7DEB781E00E94DC0539
:10095000DF91CF910895CF93DF93CDB7DEB7269780
:100960000FB6F894DEBF0FBECDBF9E838D838AE0A5
:1009700090E09C838B831CC082E390E09A83898300
:100980000EC08D819E8101979E838D838D819E8176
:100990000097B9F789819A8101979A838983898120
:1009A0009A81009799F78B819C8101979C838B8317
:1009B0008B819C81009701F726960FB6F894DEBFD5
:1009C0000FBECDBFDF91CF910895CF93DF93CDB709
:1009D000DEB721970FB6F894DEBF0FBECDBF898377
:1009E0008981992781709070882341F0A5E3B0E058
:1009F000E5E3F0E0808180618C9307C0A5E3B0E07F
:100A0000E5E3F0E080818F7E8C9389819927827065
:100A10009070009741F0A5E3B0E0E5E3F0E080815D
:100A200080628C9307C0A5E3B0E0E5E3F0E080814D
:100A30008F7D8C938981992784709070009741F005
:100A4000A5E3B0E0E5E3F0E0808180648C9307C02B
:100A5000A5E3B0E0E5E3F0E080818F7B8C938981B2
:100A6000992788709070009741F0A5E3B0E0E5E326
:100A7000F0E0808180688C9308C0A5E3B0E0E5E3F6
:100A8000F0E090818FE789238C9321960FB6F8943C
:100A9000DEBF0FBECDBFDF91CF910895CF93DF931F
:100AA000CDB7DEB7A5E3B0E0E5E3F0E08081846098
:100AB0008C9381E090E00E94AB04A5E3B0E0E5E315
:100AC000F0E080818B7F8C93DF91CF910895CF935D
:100AD000DF93CDB7DEB722970FB6F894DEBF0FBE17
:100AE000CDBF8A838A8182958F70898389810E9494
:100AF000E5040E944E058A810E94E5040E944E058D
:100B000022960FB6F894DEBF0FBECDBFDF91CF9116
:100B10000895CF93DF93CDB7DEB721970FB6F89442
:100B2000DEBF0FBECDBF8983A5E3B0E0E5E3F0E013
:100B3000808188608C9389810E94670521960FB619
:100B4000F894DEBF0FBECDBFDF91CF910895CF9354
:100B5000DF93CDB7DEB724970FB6F894DEBF0FBE94
:100B6000CDBF9C838B838B819C81DC01FD01019037
:100B70000020E9F73197CF018A1B9B0B8A831982EA
:100B80000EC0898199279C018B819C81F901E80F16
:100B9000F91F80810E94890589818F5F89839981EE
:100BA0008A81981770F324960FB6F894DEBF0FBEB3
:100BB000CDBFDF91CF910895CF93DF93CDB7DEB74F
:100BC00021970FB6F894DEBF0FBECDBF898381E0B9
:100BD00090E00E94AB04A5E3B0E0E5E3F0E08081A3
:100BE000877F8C9389810E946705A5E3B0E0E5E3E8
:100BF000F0E0808188608C9321960FB6F894DEBF78
:100C00000FBECDBFDF91CF910895CF93DF93CDB7C6
:100C1000DEB723970FB6F894DEBF0FBECDBF8A8331
:100C20006B838A81882319F48B81805889838A8118
:100C3000813019F48B818054898389810E94DC057D
:100C400023960FB6F894DEBF0FBECDBFDF91CF91D4
:100C50000895CF93DF93CDB7DEB781E090E00E9497
:100C6000AB04A5E3B0E0E5E3F0E08081877F8C93FF
:100C700083E00E94E5040E944E0585E090E00E941A
:100C8000AB0483E00E94E5040E944E0581E090E001
:100C90000E94AB0483E00E94E5040E944E0582E0BE
:100CA0000E94E5040E944E0581E090E00E94AB04A2
:100CB00088E20E94DC058EE00E94DC0581E00E9453
:100CC000DC0584E890E00E94A7056AE081E00E94CC
:100CD000050689E890E00E94A705DF91CF9108956D
:100CE000CF93DF93CDB7DEB72C970FB6F894DEBF66
:100CF0000FBECDBF8091C400882309F458C08091F5
:100D0000C700813009F051C08091C400181634F436
:100D10008091C8008F5F8093C80005C08091C80093
:100D200081508093C8008091C80088231CF483E020
:100D30008093C8008091C800843014F01092C800DD
:100D40008091C800282F332727FD30953C872B87BB
:100D50008B859C8581309105D1F02B853C85223097
:100D600031052CF48B859C85009761F01EC02B8586
:100D70003C852230310581F08B859C85833091053F
:100D800081F013C060E080E00E9405060EC069E0BB
:100D900080E00E94050609C060E081E00E9405062F
:100DA00004C069E081E00E9405061092C400E0E3FF
:100DB000F0E0808180728D838D81882361F4809141
:100DC000C700813041F48091C800823011F40E9444
:100DD000C90781E08D838D81882341F48091C7000C
:100DE000843011F40E94930781E08D838091C700C5
:100DF000843009F08FC0F8941C8217C08C81282F92
:100E000033278C819927880F991FFC01E252FF4FED
:100E1000808191819695879596958795F901EA5FEE
:100E2000FE4F80838C818F5F8C838C81863030F382
:100E300078941C826BC08C819927FC01EA5FFE4F7D
:100E4000808199279A838983CE01069629813A81E8
:100E50004AE050E0BC01C9010E94F30ECE010696A3
:100E6000DC01FD0101900020E9F73197CF018A1BD9
:100E70009B0B8B838C81843018F58C819927880F8C
:100E8000991F880F991F682F80E00E9405068EE841
:100E900090E00E94A7058C819927880F991F880FE1
:100EA000991F982F8B81292F281B822F8D5F682FE8
:100EB00080E00E940506CE0106960E94A70523C089
:100EC0008C819927880F991F880F991F8051682F4F
:100ED00081E00E9405068EE890E00E94A7058C81C3
:100EE0009927880F991F880F991F982F8B81392F69
:100EF000381B832F8D50682F81E00E940506CE019C
:100F000006960E94A7058C818F5F8C838C8186302A
:100F100008F491CF2C960FB6F894DEBF0FBECDBF6C
:100F2000DF91CF910895CF93DF93CDB7DEB781E006
:100F30008093C7001092C8000E94A10460E080E086
:100F40000E94050681E990E00E94A70569E080E023
:100F50000E94050689E990E00E94A70560E081E013
:100F60000E94050680EA90E00E94A70569E081E002
:100F70000E94050688EA90E00E94A7050E948D0461
:100F800060E080E00E9405061092C400DF91CF91DE
:100F90000895CF93DF93CDB7DEB784E08093C70089
:100FA0001092C8000E94A10469E081E00E94050639
:100FB0008FEA90E00E94A7050E948D0469E081E01D
:100FC0000E9405061092C400DF91CF910895CF933F
:100FD000DF93CDB7DEB721970FB6F894DEBF0FBE13
:100FE000CDBF1982F894E0E3F0E080819927807109
:100FF0009070009711F081E08983E0E3F0E0808158
:10100000992788709070009721F0898193E0892753
:1010100089837894998180916900292F281B822FD8
:1010200089838981992787FD9095817090708823A5
:1010300081F080916900982F8981890F80936900E0
:101040008981982F92708091C400890F815080937C
:10105000C40021960FB6F894DEBF0FBECDBFDF915E
:10106000CF910895CF93DF93CDB7DEB71092CB0029
:10107000DF91CF910895CF93DF93CDB7DEB7DF91A6
:10108000CF9108951F920F920FB60F9211242F93B4
:101090003F934F935F936F937F938F939F93AF9300
:1010A000BF93EF93FF93CF93DF93CDB7DEB72C972A
:1010B000DEBFCDBF8091CB00282F332727FD309591
:1010C0003C872B878B859C8581309105C1F02B85D2
:1010D0003C852230310529F18B859C85009709F0EC
:1010E00080C0E0E4F0E01082E9E2F0E085E0808397
:1010F000ECE2F0E0108281E08093CB0072C0E0E48B
:10110000F0E01082E9E2F0E081E08083ECE2F0E0E0
:10111000108282E08093CB001092F1001092F000D8
:1011200060C080E090E0A0E2B1E48A839B83AC835E
:10113000BD832BEA3AEA4AE250E46A817B818C81E2
:101140009D810E94B90ADC01CB018F839887A98712
:10115000BA8720E030E040E85FE36F8178858985D9
:101160009A850E94430C88230CF003C081E08E8393
:1011700018C020E030E04FE753E46F81788589851F
:101180009A850E94D70B18160CF002C01E8209C067
:101190006F81788589859A850E940809DC01CB01D9
:1011A0008E838E81898389818A95F1F78983ACE268
:1011B000B0E02091F0003091F100F901EA5FFE4FBC
:1011C00080818C93C90101969093F1008093F00087
:1011D0008091F0009091F1008233910511F410920A
:1011E000CB002C96F894DEBFCDBFDF91CF91FF915D
:1011F000EF91BF91AF919F918F917F916F915F918F
:101200004F913F912F910F900FBE0F901F90189507
:10121000EF92FF920F931F937B018C0120E030E04F
:1012200040E05FE40E940D0C88237CF020E030E079
:1012300040E05FE4C801B7010E945B0A0E94790C9C
:10124000605070408040904804C0C801B7010E94BF
:10125000790C1F910F91FF90EF900895A0E0B0E0FE
:10126000E4E3F9E00C94280FFC016A0190819230CC
:1012700008F41BC1DB018C91823080F0943061F462
:10128000843009F012C19181EB018981981709F42A
:101290000CC1E4EBF0E009C1843011F4FB0105C19D
:1012A000823091F4923009F000C1EA01DF0188E058
:1012B0000D9009928150E1F78181FB019181892391
:1012C000E6018983F601F1C0923041F362807380B8
:1012D000EB018A809B80E480F580068117812C8158
:1012E0003D814E815F815301A818B908C501B7FC43
:1012F000ABC080970CF457C0861497040CF4BEC0A2
:101300003401EE24FF2487019181FB01818198172C
:1013100009F4A6C0992309F49CC02E193F09400B7B
:10132000510B57FDB0C0E60119827B826A82F6013B
:101330002483358346835783E6012C813D814E818A
:101340005F8179018A01DA01C9010197A109B10917
:101350008F5F9F4FAF4FBF43F8F4E6016A817B81F7
:10136000A8019701220F331F441F551F6150704081
:1013700079018A01DA01C9010197A109B1098F5FD9
:101380009F4FAF4FBF4360F3E6017B836A83F60153
:10139000248335834683578383E0D6018C9357FD9E
:1013A00039C0F60182C086149704B4F4C0E0D0E0DE
:1013B000DA01C90181709070A070B07056954795A0
:1013C00037952795282B392B4A2B5B2B2196AC166A
:1013D000BD0671F78A0C9B1C681479040CF094CF3D
:1013E000C0E0D0E05401A618B708D801C701817049
:1013F0009070A070B07016950795F794E794E82A5E
:10140000F92A0A2B1B2B2196AC16BD0671F76A0C24
:101410007B1C7ACFDA01C901B695A7959795879578
:101420002170307040705070282B392B4A2B5B2B69
:10143000E6012C833D834E835F838A819B810196E5
:101440009B838A83F60131C0882799278A199B09D3
:1014500050CFE21AF30A040B150BA801970161CFD4
:10146000E60199837B826A822E0D3F1D401F511F2A
:10147000F60124833583468357838ECF20E030E006
:1014800040E050E041CF81E0E60189837B826A82BF
:1014900050954095309521953F4F4F4F5F4FF60146
:1014A000248335834683578347CFCF01EEE0CDB702
:1014B000DEB70C94440FA0E2B0E0E1E6FAE00C9451
:1014C000300F69837A838B839C832D833E834F8384
:1014D000588789E1E82EF12CEC0EFD1EB701CE01F4
:1014E00001960E94EB0D8E010F5E1F4FB801CE01D9
:1014F00005960E94EB0D8A8991E089278A8BAE01BF
:10150000475F5F4FB801C7010E942E090E94C90CB6
:10151000E6E0A0960C944C0FA0E2B0E0E2E9FAE01D
:101520000C94300F69837A838B839C832D833E8355
:101530004F83588799E1E92EF12CEC0EFD1EB7017F
:10154000CE0101960E94EB0D8E010F5E1F4FB80178
:10155000CE0105960E94EB0DAE01475F5F4FB801CB
:10156000C7010E942E090E94C90CE6E0A0960C94C7
:101570004C0FA0E2B0E0EFEBFAE00C94240F69838B
:101580007A838B839C832D833E834F8358878E0180
:10159000075E1F4FB801CE0101960E94EB0DF1E1ED
:1015A000EF2EF12CEC0EFD1EB701CE0105960E9428
:1015B000EB0D898D823078F09989923040F420E0EB
:1015C0009A8D8A89981321E02A8BB701E9C084306B
:1015D00051F4923061F020E09A8D8A89981321E0CD
:1015E0002A8FB801DDC0943029F4823041F764EBD2
:1015F00070E0D6C0823079F3923009F32D8D3E8DA4
:101600004F8D58A18D899E89AF89B88D22243324AE
:101610002101AA24BB246501EE24FF24870160E098
:1016200070E00DC06F5F7F4F6032710599F1880FD8
:10163000991FAA1FBB1F569547953795279520FFE1
:1016400019C0280E391E4A1E5B1E662477244301EA
:10165000281639064A065B0628F4E1E06E2E712C46
:10166000812C912CAE0CBF1CC01ED11EA60CB71C29
:10167000C81CD91CEE0CFF1C001F111FB7FFD2CFD6
:10168000E1E06E2E712C812C912CE628F728082998
:101690001929C8CF8B8D9C8D2B893C89820F931F74
:1016A00002969C878B871A869A8D8A89981711F0E3
:1016B00081E08A87D7FE17C08B859C85A0FE0CC071
:1016C000569447943794279420E030E040E050E867
:1016D000222A332A442A552AD694C794B794A79429
:1016E00001969C878B8730E0A31630E0B30630E08C
:1016F000C30630E4D30618F58B859C850EC0220CFA
:10170000331C441C551C019720E0A21620E0B206B1
:1017100020E0C20620E4D20680F4AA0CBB1CCC1C3C
:10172000DD1C57FEECCF31E0632E712C812C912C07
:10173000A628B728C828D928E2CF9C878B87D6014E
:10174000C5018F779070A070B07080349105A105AD
:10175000B10551F0AD86BE86CF86D88A83E08987F1
:10176000BE01675F7F4F1CC0A7FCF4CF211431047A
:101770004104510479F380E490E0A0E0B0E0A80EC9
:10178000B91ECA1EDB1E80E8682E8FEF782E8FEF01
:10179000882E8FEF982EA620B720C820D920DACF28
:1017A000CB010E94C90CE2E1A0960C94400FA8E185
:1017B000B0E0EDEDFBE00C94300F69837A838B830E
:1017C0009C832D833E834F83588781E1E82EF12C43
:1017D000EC0EFD1EB701CE0101960E94EB0D8E01AD
:1017E000075F1F4FB801CE0105960E94EB0D898956
:1017F000823018F42FEF3FEF0BC089858230D0F391
:10180000B801C7010E948A0E282F332727FD309583
:10181000C901E6E068960C944C0FA8E1B0E0E3E162
:10182000FCE00C94300F69837A838B839C832D8337
:101830003E834F83588781E1E82EF12CEC0EFD1E8C
:10184000B701CE0101960E94EB0D8E01075F1F4F7D
:10185000B801CE0105960E94EB0D8989823018F4FB
:101860002FEF3FEF0BC089858230D0F3B801C7015D
:101870000E948A0E282F332727FD3095C901E6E004
:1018800068960C944C0FA8E1B0E0E9E4FCE00C94FD
:10189000300F69837A838B839C832D833E834F83B0
:1018A000588781E1E82EF12CEC0EFD1EB701CE0128
:1018B00001960E94EB0D8E01075F1F4FB801CE010C
:1018C00005960E94EB0D8989823018F08985823057
:1018D00018F421E030E008C0B801C7010E948A0E68
:1018E000282F332727FD3095C901E6E068960C9430
:1018F0004C0FACE0B0E0EFE7FCE00C94340F6983F0
:101900007A838B839C83BE016B5F7F4FCE010196F0
:101910000E94EB0D8D81823061F0823050F0843076
:1019200069F48E81882359F52FEF3FEF4FEF5FE782
:101930002AC020E030E040E050E025C02F8138850B
:1019400037FDF7CF2F31310564F78EE190E0821B30
:10195000930B29853A854B855C8504C05695479540
:10196000379527958A95D2F78E81882361F0509517
:101970004095309521953F4F4F4F5F4F04C020E079
:1019800030E040E050E8CA01B901E2E02C960C9446
:10199000500F4F925F926F927F928F929F92AF9271
:1019A000BF92DF92EF92FF920F931F9320E030E0FF
:1019B00040E050E0FC01E480F58006811781D18091
:1019C0008081823038F4D801C701A061AF77B07050
:1019D0006FEFD9C0843009F46EC0823009F471C051
:1019E000E114F1040105110509F46BC082819381B2
:1019F0006FEF823896070CF06AC062E87FEF681BD1
:101A0000790B6A3171050CF080C047015801062E30
:101A100004C0B694A794979487940A94D2F7442468
:101A20005524320181E090E0A0E0B0E004C0880FCE
:101A3000991FAA1FBB1F6A95D2F70197A109B10987
:101A4000E822F9220A231B23E114F1040105110500
:101A500029F061E0462E512C612C712C8501740116
:101A6000E428F52806291729D801C7018F77907037
:101A7000A070B07080349105A105B10509F457C07C
:101A8000D801C701CF96A11DB11D60E070E0803084
:101A9000E0E09E07E0E0AE07E0E4BE0710F061E0A2
:101AA00070E027E0B695A795979587952A95D1F789
:101AB000AF77B07068C080E090E0A0E0B0E06FEF7A
:101AC00062C080E090E0A0E0B0E060E05CC0803800
:101AD00091058CF7BC0161587F4FD801C7018F7702
:101AE0009070A070B07080349105A105B105A1F08F
:101AF0008FE390E0A0E0B0E0E80EF91E0A1F1B1F84
:101B000017FD28C0D801C701CCCF60E070E080E0AD
:101B100090E0A0E0B0E0CCCFE7FEF2CF80E490E030
:101B2000A0E0B0E0E80EF91E0A1F1B1FE9CFE7FC9A
:101B300018C080E090E060E0E61660E0F60660E045
:101B4000060760E4160710F081E090E0BC01D801C0
:101B5000C701A7CF16950795F794E7946F5F7F4F5E
:101B6000D1CFD801C701805C9F4FAF4FBF4F60E01E
:101B700070E08030E0E09E07E0E0AE07E0E4BE0702
:101B800008F48FCF8CCF282F392F9A2F9F77842F4F
:101B90008078892B962F9795992797958F77482F3F
:101BA000492B6695852F8078862BD794DD24D79492
:101BB0008F77582F5D29CA01B9011F910F91FF90AE
:101BC000EF90DF90BF90AF909F908F907F906F903D
:101BD0005F904F900895FC01DB012081318192815B
:101BE000492F4F7750E0991F9927991F8381682FBC
:101BF000660F692B881F8827881FFD018183662354
:101C000009F049C0211531054105510509F470C09D
:101C100082E89FEFFD0193838283220F331F441FCD
:101C2000551F220F331F441F551F220F331F441F00
:101C3000551F220F331F441F551F220F331F441FF0
:101C4000551F220F331F441F551F220F331F441FE0
:101C5000551F83E08C932030F0E03F07F0E04F0702
:101C6000F0E45F0790F482E89FEF220F331F441FD8
:101C7000551F0197203060E0360760E0460760E4BA
:101C8000560798F3FD0193838283FD0124833583F6
:101C90004683578308956F3F71F1862F99278F5799
:101CA0009040FD019383828383E08C93220F331F46
:101CB000441F551F220F331F441F551F220F331F70
:101CC000441F551F220F331F441F551F220F331F60
:101CD000441F551F220F331F441F551F220F331F50
:101CE000441F551F506424833583468357830895CA
:101CF00082E08C930895211531054105510519F4B1
:101D000084E08C93089544FD02C01C92BECF81E014
:101D10008C93BBCFEF92FF920F931F93CF93DF93E0
:101D2000FC01DB018081823050F09C91923038F0D0
:101D3000843041F49430B1F08181882381F461E0F2
:101D400070E04BC09430E9F18230A1F09230A1F301
:101D50006181ED018981681791F0662381F36FEF4E
:101D60007FEF3BC0EB018981682F77278181681B5A
:101D7000710933C0923059F560E070E02EC02281C5
:101D80003381ED018A819B818217930734F32817F1
:101D900039079CF0E480F58006811781FD012481DC
:101DA0003581468157812E153F0540075107A8F21E
:101DB000E216F30604071507F8F6662309F0BFCF0D
:101DC000CECFFB018181882309F0B9CFC8CFEB01C9
:101DD0008981882309F0B3CFC2CFCB01E6E0CDB72C
:101DE000DEB70C944C0FFB019F01E8944230C4F025
:101DF0004532B4F44A3029F497FB1EF4909581954E
:101E00009F4F642F77270E945B0F805D8A330CF011
:101E1000895D8193CB010097A1F716F45DE25193A0
:101E20001082C9010C94140FDC01FC010190002008
:101E3000E9F73297AE17BF0730F47C916081708369
:101E400031976D93F7CF08952F923F924F925F9203
:101E50006F927F928F929F92AF92BF92CF92DF92BA
:101E6000EF92FF920F931F93CF93DF93CDB7DEB71F
:101E7000CA1BDB0B0FB6F894DEBF0FBECDBF0994B3
:101E80002A88398848885F846E847D848C849B840A
:101E9000AA84B984C884DF80EE80FD800C811B8118
:101EA000AA81B981CE0FD11D0FB6F894DEBF0FBE47
:101EB000CDBFED010895AA1BBB1B51E107C0AA1FAE
:101EC000BB1FA617B70710F0A61BB70B881F991FDB
:0E1ED0005A95A9F780959095BC01CD01089513
:101EDE004B2000000000003D00010D0A4550492D29
:101EEE005465737465720056657273696F6E203037
:101EFE002E3264006875687500416B6B750020208A
:101F0E000050504D2D4F75740050504D2D496E00A0
:101F1E00444D582D4F757400444D582D496E004553
:0C1F2E0078697400000000000000000052
:00000001FF
